:10000000B201BC290408A20083160710831209302C
:10001000A30003101220A20CA30B0A280314122021
:100020000314B7290318172800000714192807100C
:1000300019280030A10062306029B216B21EB21237
:10004000B2192628B2155F2003184D280830A300E6
:100050007320A20DA30B2828B21E58207D207920E2
:10006000B21A4D20522022080310B729B216B21E30
:10007000B21232194028FE39B30032150310B729E5
:10008000321A4828A60032165F2003184D28260889
:10009000662003184D28B21EB72958207D20321142
:1000A0003212B211360884003408841780045E28A6
:1000B0003608840034098005841780050800522022
:1000C0007D20582079203308B2190138A200083069
:1000D000A300A20D03185220031C58207D20792074
:1000E000A30B692852207D203608840034080005BF
:1000F000FF3E3708840035095B283708840035083F
:1001000055282C08A0002D08A1000130A200A30151
:100110006400AF20031C9C28A20B8828FF30A30793
:1001200003188828A007031CA107031C08006430DB
:10013000A2000030A30088280221A8010830A300F3
:100140000321AF200318A80AAB1EA801A20CA30B21
:10015000A028AB1AA21303210314220808003608B2
:100160008400340884178004841300052B1B340694
:10017000FF3E0800A400290803140319B729B2217F
:10018000031C0800A00025188317240884002008F9
:1001900080008313A40AA903BB280408A60036081C
:1001A00084008030B3050830A70003100318B30A99
:1001B000E820A60CA70BD6280000AB1A330CE820C9
:1001C000BA210314E8202F08A3002E085321B729D1
:1001D0008413AB1FF728000834042B1F340680005B
:1001E000841700083404031C340680000329000827
:1001F0003404031C34062B1B340680008417340996
:100200008005032933172B081F39003EA1002A0857
:10021000043E0318A10A331F60293313A000031002
:10022000A10CA00C0310A10C200C6029A40029082B
:100230000319B7292518831724088400000883139D
:10024000B221A40AA9031829B31329080319B31763
:100250000530A8002730A30010303A210330A30056
:10026000E8303A21A30164303A21A3010A303A214F
:1002700024084129A2002508A1002408A0009621F5
:100280002008A000A8030319B313290803194B2958
:100290002802031808002008031DB313B31B08002D
:1002A000303EB229A301A200FF30A207031CA3071E
:1002B000031CB7290330A100E33060215429A101B8
:1002C000F43EA000A109FE30031C6929A007031811
:1002D0006629A0076400A10F662900002018702974
:1002E0002018722908000310A00DA10DFF3E03186D
:1002F00073292008B7290310A10CA00CFF3E031896
:100300007B292008B729A20004308629A8002308E9
:100310002102031D8D292208200204300318013018
:10032000031902302805031DFF30B729A501A401D8
:100330001030A600210DA40DA50D2208A40223084B
:10034000031C230FA5020318AC292208A4072308C5
:100350000318230FA5070310A00DA10DA60B9A29C2
:100360002008B729840031088A00300882008313EE
:100370000313831264000800831671308F00071185
:1003800005150710051485148516871105123030E0
:100390009F000630910083129901051683160512FD
:1003A0008312E401E501DE01DF0156308A010320FA
:1003B00044308A01032072308A01032069308A01A7
:1003C000032076308A01032065308A010320323011
:1003D0008A01032020308A01032053308A01032040
:1003E00054308A01032041308A01032052308A01AF
:1003F000032054308A01032049308A0103204E3003
:100400008A01032047308A0103200D308A0103202E
:100410000A308A010320C8308A0152210716831648
:10042000071283120230A30058308A01532153303F
:100430008A01032059308A0103204E308A010320AB
:1004400043308A01032048308A01032052308A0158
:1004500003204F308A0103204E308A0103204930A7
:100460008A0103205A308A01032049308A0103207F
:100470004E308A01032047308A0103200D308A0163
:1004800003200A308A010320FA308A0152215330B6
:100490008A01032065308A0103206E308A0103201F
:1004A00064308A01032069308A0103206E308A019A
:1004B000032067308A01032020308A010320453061
:1004C0008A0103200D308A0103200A308A010320AB
:1004D0000730B6001030B4005430AA00AB01AE01B2
:1004E000AF0145308A01CE200D308A01CE20073081
:1004F000B6002030B4005430AA00AB016430AC0028
:10050000AD018A0181208A11031CB02AE800533012
:100510008A01032065308A0103206E308A0103209E
:1005200074308A01032020308A01032045308A017B
:1005300003203D308A01032020308A01032068080F
:100540008A0103200D308A0103200A308A0103202A
:1005500064006808453C8A110319DF2A8A01442A8D
:100560004E308A0103206F308A01032020308A0137
:10057000032045308A01032020308A010320723095
:100580008A01032065308A01032074308A01032028
:1005900075308A01032072308A0103206E308A018F
:1005A000032065308A01032064308A0103200D3066
:1005B0008A0103200A308A0103208A01442A533029
:1005C0008A01032065308A0103206E308A010320EE
:1005D00064308A01032020308A01032053308A01CD
:1005E000032055308A01032044308A0103200D3056
:1005F0008A0103200A308A0103200730B600103038
:10060000B4005430AA00AB01AE01AF0153308A01EF
:10061000CE2055308A01CE2044308A01CE200D30C4
:100620008A01CE200730B6001030B4005430AA0042
:10063000AB01AE01AF0152308A01CE2044308A01B5
:10064000CE2020308A01CE2064308A01CE20613055
:100650008A01CE2074308A01CE2065308A01CE20F6
:100660002E308A01CE2074308A01CE2078308A0163
:10067000CE2074308A01CE200D308A01CE20073082
:10068000B6002030B4005430AA00AB015830AC00A2
:100690000230AD000E30A9008130B000B101A501DB
:1006A00038308A01BA208A11031C152D64003808DD
:1006B000433C8A110319152D64308A0103206130EF
:1006C0008A01032074308A01032065308A010320E7
:1006D00073308A01032074308A01032072308A014A
:1006E000032069308A0103206E308A0103206730BD
:1006F0008A0103203D308A01032020308A01032033
:100700000E30A9000230B000B101A50138308A01D5
:1007100016210D308A0103200A308A01032073302C
:100720008A01032065308A01032074308A01032086
:1007300063308A0103206C308A0103206F308A0104
:10074000032063308A0103206B308A0103200D30BF
:100750008A0103200A308A010320F201D0304507C4
:10076000E000FF300318013EE100D0304407E20012
:10077000FF300318013EE3006208A0006308A100F7
:1007800004308A017621E2002108E3006008620754
:10079000F000D0304207E000FF300318013EE100D6
:1007A000D0304107E200FF300318013EE300620849
:1007B000A0006308A10004308A017621E20021082C
:1007C000E30060086207EF00F301D0303F07E0006C
:1007D000FF300318013EE100D0303E07E200FF3059
:1007E0000318013EE3006208A0006308A100043082
:1007F0008A017621E2002108E30060086207EE002A
:10080000D0303C07E000FF300318013EE100D0305B
:100810003B07E200FF300318013EE3006208A0003E
:100820006308A10004308A017621E2002108E30078
:1008300060086207F100D0303907E000FF3003188C
:10084000013EE100D0303807E200FF300318013EDE
:10085000E3006208A0006308A10004308A01762149
:10086000E2002108E30060086207F4001030ED00A8
:100870000730B6000830B4000730B7000430B500C8
:10088000D0308A01382000308A01382072088A016D
:10089000382070088A0138206F088A0138207308D0
:1008A0008A0138206E088A01382071088A013820B0
:1008B00074088A0138206D088A01362064308A0164
:1008C00052210730B6001030B4005430AA00AB01FA
:1008D000AE01AF0152308A01CE2045308A01CE20D0
:1008E0004E308A01CE2020308A01CE2064308A0129
:1008F000CE2061308A01CE2074308A01CE2065304E
:100900008A01CE202E308A01CE2074308A01CE207A
:1009100078308A01CE2074308A01CE2020308A01BE
:10092000CE206E308A01CE2064308A01CE20613024
:100930008A01CE2074308A01CE2065308A01CE2013
:100940002E308A01CE2074308A01CE2078308A0180
:10095000CE2074308A01CE200D308A01CE20723034
:100960008A01032065308A0103206E308A0103204A
:1009700061308A0103206D308A01032065308A01CD
:10098000032020308A01032064308A010320613073
:100990008A01032074308A01032065308A01032014
:1009A0002E308A01032074308A01032078308A01B6
:1009B000032074308A01032020308A010320743020
:1009C0008A0103206F308A01032020308A0103202E
:1009D0006E308A01032064308A01032061308A016D
:1009E000032074308A01032065308A0103202E30F1
:1009F0008A01032074308A01032078308A010320A1
:100A000074308A01032020308A0103200E30A900AF
:100A10000230B000B101A50138308A0116210D3035
:100A20008A0103200A308A0103208A15A0208A1532
:100A30006E2164008A11851E2B2D8A1553220330E6
:100A4000A300E8308A0153210512831605126400C1
:100A500083128A01272D0330A30020308A015321FD
:100A60008A11E9278A110E268A113D268A116C26E1
:100A700053308A01032074308A01032065308A01D3
:100A8000032070308A01032020308A010320A9014D
:100A90005E08A4005F08A5000230B000B1018A0121
:100AA000242120308A01032046308A010320693046
:100AB0008A0103206C308A01032065308A010320FB
:100AC0003A308A01032020308A010320A90152080C
:100AD000A400A5010230B000B1018A012421A901BE
:100AE0005308A400A5010230B000B1018A012421FD
:100AF000A9015408A400A5010230B000B1018A0187
:100B00002421A9015508A400A5010230B000B101BB
:100B10008A012421A9015608A400A5010230B000D1
:100B2000B1018A012421A9015708A400A5010230BE
:100B3000B000B1018A012421A9015808A400A5012F
:100B40000230B000B1018A012421A9015908A40092
:100B5000A5010230B000B1018A0124212E308A01A2
:100B6000032063308A01032073308A01032076302A
:100B70008A0103200D308A0103200A308A010320F4
:100B800054308A01032069308A0103206D308A01C4
:100B9000032065308A01032020308A010320A90147
:100BA0006A08A400A5010230B000B1018A01242125
:100BB000A9016908A400A5010230B000B1018A01B1
:100BC00024213A308A010320A9017D08A400A5014F
:100BD0000230B000B1018A012421A9017C08A400DF
:100BE000A5010230B000B1018A0124210D308A0133
:100BF00003200A308A0103205E08A0005F08A100DC
:100C00001C30A30021308A0183218A11031D192D74
:100C10008A155322DE01DF018A01152D85309F00E0
:100C20009F1464308A015F211E08DB0083161E08B2
:100C30008312DA0041308A01032044308A01032004
:100C400043308A01032031308A0103203D308A017C
:100C5000032020308A010320A9015A08A4005B0860
:100C6000A5000230B000B1018A0124210D308A01B3
:100C700003200A308A010320080089309F009F1456
:100C800064308A015F211E08DD0083161E0883126E
:100C9000DC0041308A01032044308A0103204330C4
:100CA0008A01032032308A0103203D308A0103206B
:100CB00020308A010320A9015C08A4005D08A5007A
:100CC0000230B000B1018A0124210D308A010320D5
:100CD0000A308A0103200800DE0A0319DF0A5730B0
:100CE0008A01032072308A01032069308A010320BF
:100CF00074308A01032065308A01032020308A0184
:100D00000320A901831622088312A400A501023042
:100D1000B000B1018A012421A901831621088312A0
:100D2000A400A5010230B000B1018A012421A9016B
:100D30006C08A400A5010230B000B1018A01242191
:100D4000A9016B08A400A5010230B000B1018A011D
:100D50002421A9016708A400A5010230B000B10157
:100D60008A012421A9016608A400A5010230B0006F
:100D7000B1018A012421A9016A08A400A501023059
:100D8000B000B1018A012421A9016908A400A501CC
:100D90000230B000B1018A012421A9017D08A4001C
:100DA000A5010230B000B1018A012421A9017C080B
:100DB000A400A5010230B000B1018A012421A901DB
:100DC0007F08A400A5010230B000B1018A012421EE
:100DD000A9017E08A400A5010230B000B1018A017A
:100DE00024212C308A0103200430A9005A08A400D1
:100DF0005B08A5000230B000B1018A0124212C302B
:100E00008A0103200430A9005C08A4005D08A50045
:100E10000230B000B1018A0124210D308A01032083
:100E20000A308A0103200730B6001030B400543075
:100E3000AA00AB01AE01AF0157308A01CE2052307B
:100E40008A01CE2046308A01CE2020308A01CE2071
:100E500000308A01CE2000308A01CE2000308A0185
:100E6000CE2017308A01CE200D308A01CE20A90174
:100E7000831622088312A400A501CD30B000B10171
:100E80008A012421A901831621088312A400A50147
:100E9000CD30B000B1018A012421A9016C08A40061
:100EA000A501CD30B000B1018A012421A9016B0850
:100EB000A400A501CD30B000B1018A012421A9010F
:100EC0006708A400A501CD30B000B1018A0124213A
:100ED000A9016608A400A501CD30B000B1018A01C6
:100EE0002421A9016A08A400A501CD30B000B101F8
:100EF0008A012421A9016908A400A501CD30B00010
:100F0000B1018A012421A9017D08A400A501CD30E9
:100F1000B000B1018A012421A9017C08A400A50127
:100F2000CD30B000B1018A012421A9017F08A400BD
:100F3000A501CD30B000B1018A012421A9017E08AC
:100F4000A400A501CD30B000B1018A0124212C30CC
:100F50008A01CE200430A9005A08A4005B08A5002D
:100F6000CD30B000B1018A0124212C308A01CE207D
:100F70000430A9005C08A4005D08A500CD30B000D5
:100F8000B1018A0124210D308A01CE200D308A0161
:100F9000CE20080046308A01032061308A010320F8
:100FA00069308A0103206C308A01032020308A01D5
:100FB000032049308A01032032308A010320433064
:100FC0008A0103200D308A0103200A308A010320A0
:100FD000080052308A01032065308A010320613005
:100FE0008A01032064308A01032020308A01032013
:100FF00052308A01032054308A01032043308A0191
:1010000003200D308A0103200A308A0103200730B3
:10101000B6000830B4000730B7000430B500D03057
:101020008A0138208A110318CA2F00308A0138201B
:101030008A110318CA2F8A011F208A110318CA2F88
:10104000F2008A011F208A110318CA2FF0008A01BA
:101050001F208A110318CA2FEF008A011F208A114E
:101060000318CA2FF3008A011F208A110318CA2F00
:10107000EE008A011F208A110318CA2FF1008A018D
:101080001F208A110318CA2FF4008A011D208A111B
:101090000318CA2FED000F307205FE007030720584
:1010A000FF007F08A000A10104308A017E21FF001B
:1010B0000F307005FC0070307005FD007D08A00049
:1010C000A10104308A017E21FD000F306F05E90087
:1010D00030306F05EA006A08A000A10104308A01DF
:1010E0007E21EA000F306E05E60030306E05E70025
:1010F0006708A000A10104308A017E21E7000F30BB
:101100007105EB0010307105EC006C08A000A10126
:1011100004308A017E21EC000F3074058316A10093
:10112000F030831274058316A20022088312A000F7
:10113000A10104308A017E218316A20083120800D7
:101140004D308A0103204B308A01032020308A0170
:10115000032066308A01032069308A0103206C3045
:101160008A01032065308A01032020308A01032090
:101170006E308A01032061308A0103206D308A01BC
:10118000032065308A01032020308A010320733058
:101190008A01032074308A01032072308A010320FF
:1011A00069308A0103206E308A01032067308A018A
:1011B00003200D308A0103200A308A010320073002
:1011C000B6000830B4000730B7000430B500D030A6
:1011D0008A0138208A110318CA2F00308A0138206A
:1011E0008A110318CA2F8A011F208A110318CA2FD7
:1011F000F2008A011F208A110318CA2FF0008A0109
:101200001F208A110318CA2FEF008A011F208A119C
:101210000318CA2FF3008A011F208A110318CA2F4E
:10122000EE008A011F208A110318CA2FF1008A01DB
:101230001F208A110318CA2FF4008A011D208A1169
:101240000318CA2FED000F306F05E9006908D900B7
:1012500030306F05EA006A08A000A10104308A015D
:101260007E21EA006A08D8000F306E05E6006608A5
:10127000D70030306E05E7006708A000A1010430F8
:101280008A017E21E7006708D6000F307105EB0068
:101290006B08D50010307105EC006C08A000A101AE
:1012A00004308A017E21EC006C08D4000F307405F4
:1012B0008316A10021088312D300F0307405831631
:1012C000A20022088312A000A10104308A017E211D
:1012D0008316A20022088312D20008000730B6004D
:1012E0001030B4005430AA00AB01AE01AF014F3052
:1012F0008A01CE2050308A01CE2057308A01CE207C
:1013000020308A01CE20A9015208A400A501CD30C9
:10131000B000B1018A012421A9015308A400A5014C
:10132000CD30B000B1018A012421A9015408A400E4
:10133000A501CD30B000B1018A012421A9015508D1
:10134000A400A501CD30B000B1018A012421A9017A
:101350005608A400A501CD30B000B1018A012421B6
:10136000A9015708A400A501CD30B000B1018A0140
:101370002421A9015808A400A501CD30B000B10175
:101380008A012421A9015908A400A501CD30B0008B
:10139000B1018A0124212E308A01CE2063308A01D6
:1013A000CE2073308A01CE2076308A01CE200D30D7
:1013B0008A01CE204F308A01032070308A01032039
:1013C00065308A0103206E308A01032020308A01B3
:1013D000032066308A01032069308A0103206C30C3
:1013E0008A01032065308A01032020308A0103200E
:1013F000A9015208A400A5010230B000B1018A0180
:101400002421A9015308A400A5010230B000B101B4
:101410008A012421A9015408A400A5010230B000CA
:10142000B1018A012421A9015508A400A5010230B7
:10143000B000B1018A012421A9015608A400A50128
:101440000230B000B1018A012421A9015708A4008B
:10145000A5010230B000B1018A012421A901580878
:10146000A400A5010230B000B1018A012421A90124
:101470005908A400A5010230B000B1018A0124215D
:101480002E308A01032063308A01032073308A01E1
:10149000032076308A0103200D308A0103200A30B0
:1014A0008A01032008000730B6001030B400543021
:1014B000AA00AB01AE01AF0143308A01CE204C300F
:1014C0008A01CE2046308A01CE2020308A01CE20EB
:1014D000A9015208A400A501CD30B000B1018A01D4
:1014E0002421A9015308A400A501CD30B000B10109
:1014F0008A012421A9015408A400A501CD30B0001F
:10150000B1018A012421A9015508A400A501CD300B
:10151000B000B1018A012421A9015608A400A50147
:10152000CD30B000B1018A012421A9015708A400DF
:10153000A501CD30B000B1018A012421A9015808CC
:10154000A400A501CD30B000B1018A012421A90178
:101550005908A400A501CD30B000B1018A012421B1
:101560002E308A01CE2063308A01CE2073308A016A
:10157000CE2076308A01CE200D308A01CE20433035
:101580008A0103206C308A0103206F308A01032016
:1015900073308A01032065308A01032020308A01DC
:1015A000032066308A01032069308A0103206C30F1
:1015B0008A01032065308A01032020308A0103203C
:1015C000A9015208A400A5010230B000B1018A01AE
:1015D0002421A9015308A400A5010230B000B101E3
:1015E0008A012421A9015408A400A5010230B000F9
:1015F000B1018A012421A9015508A400A5010230E6
:10160000B000B1018A012421A9015608A400A50156
:101610000230B000B1018A012421A9015708A400B9
:10162000A5010230B000B1018A012421A9015808A6
:10163000A400A5010230B000B1018A012421A90152
:101640005908A400A5010230B000B1018A0124218B
:101650002E308A01032063308A01032073308A010F
:10166000032076308A0103200D308A0103200A30DE
:101670008A01032008000A308A0103200A308A0107
:10168000032062308A01032061308A010320643024
:101690008A0103205F308A01032064308A0103201D
:1016A00061308A01032074308A01032061308A018D
:1016B000032063008A15592B49308A0103204430E6
:1016C0008A01032020308A01032065308A0103202B
:1016D00072308A01032072308A0103206F308A0140
:1016E000032072308A0103200D308A0103200A3062
:1016F0008A01032064008A157A2B44308A01032072
:101700004F308A0103204E308A01032045308A0180
:1017100003200D308A0103200A308A0103200512BC
:0C17200083160512640083128A15922BB8
:02400E00FC3F75
:00000001FF
